:02000000B22B21
:1000080070082000A00080318B1E24280B1D242896
:1000180095012100A20A0319A30A2308003C031D25
:100028001828220820004902031823282100A201C9
:10003800A301200095010130ED000030EE000B1106
:0800480020002008F00009006F
:100050002400141935281F301605F1007108003AE4
:0E006000031D35280130F0003628F00108009D
:10006E00200091112200640824009100141D4028E4
:10007E003D2820009119442840282400161B4928A9
:0C008E00F0014C2816150230F0000800AC
:10009A002200E401E5016508123C031D56286408A4
:1000AA008E3C031C62282820700803195D286228E8
:1000BA002200E40A0319E50A5028220012306502D8
:1000CA00031D69288F306402031C6E287B30F00000
:1000DA00742824001614161C73287028F0010800CE
:0600EA00240016150800B9
:1000F00023009E187D280000782822006008230035
:040100009A00080059
:100104002200E301F0306005E1006008E200E2351E
:10011400E235E235E235F030E2054D2028204E305C
:100124002200E40037202820220063086104E40050
:100134006415E415372028204230FD00FD0BA0286B
:100144000000220063086104E400E415372028203D
:100154008530FD00FD0BAC28220063086204E40036
:100164006415E415372028204230FD00FD0BB82823
:100174000000220063086204E400E415372028200C
:10018400752022006008013A031DD1280B30FC00C1
:100194006230FD00FD0BCC28FC0BCC2800000800CD
:1001A4002000F801F9011030FC00710DF80DF90D73
:1001B4007408F8027508031C750FF9020318E9287E
:1001C4007408F80775080318750FF9070310F00D84
:0801D400F10DFC0BD728080017
:1001DC002000F8010830FC00700DF80D7408F802CE
:1001EC000318FA28F8070310F00DFC0BF22808008E
:1001FC0001302200DF001E295B03F0007008803EF6
:10020C00E00082202E295B03F0007008C03EE00065
:10021C0082202E295B03F0007008943EE0008220BF
:10022C002E295B03F0007008D43EE00082202E29BA
:10023C005A08013A031902295A08023A03190929E2
:10024C005A08033A031910295A08043A03191729B2
:10025C00F0305C05DD005C08DE00DE35DE35DE35B9
:10026C00DE35F030DE054D2028204E302200E40033
:10027C003720282022005F085D04E4006415E41593
:10028C00372028204230FD00FD0B4A2900002200B7
:10029C005F085D04E400E415372028208530FD005C
:1002AC00FD0B562922005F085E04E4006415E4157A
:1002BC00372028204230FD00FD0B6229000022006F
:1002CC005F085E04E400E415372028207520080040
:0A02DC0071088A0070088200080013
:1002E6002100151595141514951195120B118B12E5
:0802F600200095019E010800A3
:1002FE0024001413941321000C158C143830240090
:04030E00950008004E
:100312002200D601540884005508850000082100F7
:10032200EF006F08003A0319A6296F082200E000C7
:1003320078202200D60A5608540784000030553D22
:0C034200850000082100EF00922908004F
:10034E00220054088400550885000008F00070084B
:10035E000319BD2954088400550885000008E000E3
:0E036E0078202200D40A0319D50AA729080016
:10037C00FF302200A800FF30A900FF30AA00FF3098
:0E038C00AB00F03021009E009D011D14080002
:10039A002200560884005708850000080319E62938
:1003AA005408DA005508DB0056088400570885000F
:1003BA000008DC00FE202200D50AD60A0319D70A53
:0403CA00CD29080031
:1003CE0012001E00F003031DE729F103031DE729A8
:0203DE00080015
:1003E00078302200A4000030A5006030A600013063
:1003F000A700FF30A000FF30A1000030A2000030B5
:10040000A300FF30B000FF30B1000030B200003078
:10041000B300FF30AC00FF30AD000030AE00003064
:10042000AF0023009E1690309D0021008C140C1408
:100430002000911E1F2A23001908F000182A080026
:100440002100EF0103306F020318322A6F082200E7
:10045000550786000030563D87002030810021007E
:10046000EF0A222A6F082200550786000030563D09
:10047000870081012100EF036F0822005507D70094
:100480000030563DD8000A30F4005408F000EE2049
:100490007808F0003030F00722005708860058082E
:1004A0008700700881000A30F4005408F000EE2044
:1004B00070082200D4007008003A031D602A632AE5
:0804C0002100EF033C2A0800B3
:1004C8002100EF0105306F020318762A6F08220019
:1004D800560786000030573D8700203081002100F4
:1004E800EF0A662A6F082200560786000030573D3B
:1004F800870081012100EF036F0822005607D8000A
:100508000030573DD9000A30F400F5015408F000D6
:100518005508F100D2207808F0007908F100303051
:10052800F0072200580886005908870070088100E3
:100538000A30F400F5015408F0005508F100D22003
:1005480070082200D4007108D50000307106031D20
:10055800AF2A00307006031DB22AB52A2100EF0326
:04056800802A0800DD
:10056C002100EF014D2028204E302200E4003720DE
:10057C0028209C30FC00D730FD00FD0BC32AFC0B5F
:10058C00C32A303021006F042200E4006415E41506
:10059C00372028204230FD00FD0BD22A00003030DD
:1005AC0021006F042200E400E415372028203430A9
:1005BC00FC00F130FD00FD0BE12AFC0BE12A0000F0
:1005CC000000303021006F042200E4006415E415B3
:1005DC00372028204230FD00FD0BF22A000030307D
:1005EC0021006F042200E400E41537202820343069
:1005FC00FC00F130FD00FD0B012BFC0B012B00006E
:10060C000000303021006F042200E4006415E41572
:10061C00372028204230FD00FD0B122B000030301B
:10062C0021006F042200E400E41537202820343028
:10063C00FC00F130FD00FD0B212BFC0B212B0000ED
:10064C000000203021006F042200E4006415E41542
:10065C00372028204230FD00FD0B322B00002030CB
:10066C0021006F042200E400E415372028207520B7
:10067C003430FC00F130FD00FD0B422BFC0B422B07
:10068C000000000028302200E00082200630E0004C
:04069C0082200800B0
:1006A0002200B4012100A401A501B101B201A601FB
:1006B000A701F101F20180307206F0008030700273
:1006C000031D642B203071020318712B3430710725
:1006D00086000130723D87008101F10A0319F20A98
:1006E0005B2B23001908F100F2012100911608008C
:1006F00022002608860021006F088100860A220059
:0C0700002408F0002508F1006E2108001C
:10070C000D302200E00078200A302200E000782032
:02071C000800D3
:10071E00220056088400570885000008F000700873
:10072E000319AC2B56088400570885000008F0000A
:10073E00540886005508870070088100D40A0319F2
:10074E00D50AD60A0319D70A8F2B540886005508E6
:06075E0087008101080084
:1007640090277830210099002F308C0023008C01D1
:100774000C14303024008C002200910192019D0160
:100784009D149D171D15243021008C0020000C1091
:100794002200971797121716971117119714171409
:1007A4005023B330DB000030DC0023009F15CF3032
:1007B4009B009C011E15F0212000911EE52B2300B7
:1007C40019082100AA002000911EEC2B230019080F
:1007D4002100AA000B30FB002630FC005D30FD0038
:1007E4002100FD0BF22BFC0BF22BFB0BF22B000078
:1007F40000000C30EF0078238B012000910192015E
:100804000B118B160B138B132100AB01AC01A80148
:10081400A901A401A5010C302200E00078200B30CE
:10082400FB002630FC005D30FD00FD0B172CFC0B9B
:10083400172CFB0B172C0000000041302200E000B5
:10084400782042302200E000782043302200E0008B
:1008540078202100A601A701B101B2018623B3309B
:100864002100DB000030DC005B082200D400210002
:100874005C082200D5008930D6008630D7008F234B
:10088400B3302100DB000030DC005B082200D40020
:1008940021005C082200D50089215B082200D400D5
:1008A40021005C082200D5001B30D6008730D70019
:1008B4008F23B3302100DB000030DC005B08220012
:1008C400D40021005C082200D50089215B082200A5
:1008D400D40021005C082200D500B530D600863053
:1008E400D7008F23B3302100DB000030DC005B082D
:1008F4002200D40021005C082200D50089215B0875
:100904002200D40021005C082200D500DC30D6008F
:100914008630D7008F23B3302100DB000030DC00A9
:100924005B082200D40021005C082200D500892144
:100934008623B3302100DB000030DC008623210055
:10094400AD01AE01AF01B001AA0123009D011D1646
:100954009D179D1619082100AA00BE219E141E147D
:100964009E139D011D111D14FE302200D4008630FB
:10097400D500A7212100A201A3012000ED01EE0171
:1009840095017321950174302200D4008730D5007D
:10099400A7210B118B166130D4008730D500A72115
:1009A4002830240092007F2183302200D400873035
:1009B400D500A721B6220C30E00082200130E000EF
:1009C40082200130D4000130D5002130D60000301F
:1009D400D700CD213830D4008730D500A721862315
:1009E4002100A401A501AB01AC01A801A9012000CB
:1009F400EB01EC01E901EA012100A001A1012000C1
:100A0400ED01EE010B178B17B3302100DB00003032
:100A1400DC0021082200D40021005B082200D5005C
:100A240021005C082200D600202221005B0822005D
:100A3400D40021005C082200D5008921093022005D
:100A4400E000782001302200D4000130D5003B3092
:100A5400D6000030D700CD210130D4000D30D500B0
:100A640021005B082200D60021005C082200D70088
:100A7400CD2121009D149D1C402D3D2D1C082000DE
:100A8400EF006F082200D40021005B082200D5008B
:100A940021005C082200D600202202302200D4006B
:100AA4000130D5003630D6000030D700CD210230D9
:100AB400D4000530D50021005B082200D6002100B7
:100AC4005C082200D700CD2121005B082200D4005D
:100AD40021005C082200D500892109302200E000B1
:100AE4007820DD3086000030870021002108860749
:100AF4000318870A20006F0881002100A10A20083A
:100B0400013A031D182E2000EB01EC012100ED0138
:100B1400EE0100306E02031D912D10306D0203189A
:100B2400A62DDD306D07840000306E3D8500000881
:100B3400F000F10170082000EB077108EC3D210082
:100B4400ED0A0319EE0A8B2D20006B082200D40055
:100B540020006C082200D50021005B082200D6008A
:100B640021005C082200D700642203302200D40054
:100B74000130D5004F30D6000030D700CD210330EE
:100B8400D4000530D50021005B082200D6002100E6
:100B94005C082200D700CD2121005B082200D4008C
:100BA40021005C082200D500892109302200E000E0
:100BB400782020006B08F0006C08F100F136F00C8E
:100BC400F136F00CF136F00CF136F00C7008E90057
:100BD40004302200D4000130D5004A30D600003061
:100BE400D700CD210430D4000530D50021005B08A6
:100BF4002200D60021005C082200D700CD2120006D
:100C040069082200D40021005B082200D5002100DD
:100C14005C082200D600202221005B082200D400B8
:100C240021005C082200D5008921272E4E302200A5
:100C3400D4008730D500A7210130D4000130D5007D
:100C44005430D6000030D700CD21210021080F3CBC
:100C540003182F2E0130A000A101862300302000AC
:100C64006E06031D372E00306D06031D3A2E302EFE
:080C7400ED01EE01062D3D2EFD
:100F200041308400863085004830F0000130F10007
:0C0F30002130860000308700E721080017
:100C820049343234433420344C34433444343434DD
:100C92007834323430342C34553441345234543470
:0A0CA2002C34413444344334003450
:0A0CAC004E346F3477343D340034C9
:100CB60049346E34643465347834203446344934E7
:0C0CC6004C344F3420343D3420340034D2
:020CD2001E34CE
:0A0CD4004D346F3479343D340034A0
:0A0CDE00533475346D343D34003496
:100CE80057346134693474342034463469346C348C
:100CF80074346534723469346E3467342034203483
:0A0D0800203420342034203400345D
:100D120054346534733474342034493432344334B3
:100D220020344C3443344434343478343234303420
:100D320020342B342034413444344334203461345D
:100D420076346534633420346D346F34793420342E
:100D520067346C3469347334733461346E3474348C
:080D620065340D340A3400343D
:100D6A00563465347234733469346F346E342034D3
:100D7A00313434342F34303436342F34323430343E
:100D8A00313435342034203420344D3469346B34D2
:100D9A0072346F3443342034503472346F34203414
:0E0DAA0036342E34353430340D340A340034EF
:100DB8005534413452345434203431343934323493
:100DC800303430342034203446344F3453344334B0
:100DD800203469346E347434653472346E34653456
:100DE80020342034313436344D3468347A340D3478
:040DF8000A34003485
:100DFC00493454342034553441345234543420342E
:100E0C005234413434342D3452344134353420345A
:100E1C0026342034543469346D34653472343034AF
:0A0E2C00203420340A340D34003461
:100E36003134323446343134383434343034203476
:100E460020346134763465346334203469346E3446
:100E560074346534723466346134633465342034F2
:0A0E6600323454340D340A340034E1
:100E70004C34433444342034493432344334203401
:100E8000343478343234303420342E342E346934CF
:0C0E90006E34693474340D340A340034BC
:100E9C00203420345734613469347434203466344B
:100EAC0069346C3474346534723469346E34673438
:060EBC002E342E34003438
:100EC20049346E3469347434203469346E34743481
:100ED2006534723472347534703474342E342E3472
:060EE2000D340A34003457
:100EE80049346E34693474342034543469346D347C
:0E0EF80065347234303420340A340D34003442
:100F0600493432344334203469346E3469347434A9
:080F16002E340D340A340034BE
:020000040001F9
:04000E00840913341A
:020000040001F9
:10E000004D0065007300750072006500200064001B
:10E010006500200044006500620069007400200073
:10E0200020004500610075002000410064006F0081
:10E03000750063006900730073006500750072006D
:10E04000430075006C006C006900670061006E00A1
:10E0500020000D000A000000FF00FF00FF00FF008D
:10E0600050004900430031003200460031003800C2
:10E070003400300020002B00200049006E007400A6
:10E0800066006100630065002000630061007000AD
:10E0900074006500750072002000640065002000B7
:10E0A0002000640065006200690074000D000A0031
:10E0B0000000FF00FF00FF00FF00FF00FF00FF0067
:10E0C0004D0069006B0072006F004300200050009B
:10E0D00072006F00200036002E0034003000200057
:10E0E000200072006500670069007300740065001D
:10E0F0007200650064000D000A00000000000000CE
:10E10000FF00FF00FF00FF00FF00FF00FF00FF0017
:10E11000FF00FF00FF00FF00FF00FF00FF00FF0007
:10E12000FF00FF00FF00FF00FF00FF00FF00FF00F7
:10E13000FF00FF00FF00FF00FF00FF00FF00FF00E7
:10E1400049006E0069007400200048004300300060
:10E150003600200042006C006500750000000000E1
:10E16000FF00FF00FF00FF00FF00FF00FF00FF00B7
:10E17000FF00FF00FF00FF00FF00FF00FF00FF00A7
:10E18000FF00FF00FF00FF00FF00FF00FF00FF0097
:10E19000FF00FF00FF00FF00FF00FF00FF00FF0087
:10E1A0002A00FF00FF00FF00FF00FF00FF00FF004C
:10E1B000FF00FF00FF00FF00FF00FF00FF00FF0067
:10E1C0007000610075006C0066006A0075006A00EE
:10E1D0006F002E0066007200650065002E0066006C
:10E1E00072000D000A000000FF00FF00FF00FF00AA
:10E1F000FF00FF00FF00FF00FF00FF00FF00FF0027
:00000001FF
